:020000040000FA
:020000001B28BB
:08000800B000030EB100C40BAF
:1000100015284008B2004108B300C6203208C000CD
:100020003308C100C301C30AC320310E8300B00EE0
:10003000300E0C100900831603137C308F008113DF
:100040001B1400009B148501051400008514860113
:10005000831203138B0107309C0081309F008316AD
:1000600003139F01831603138C010C1483120313D3
:10007000EA308F0060308E000B1700008B1738308D
:1000800090001014C3204B202108A000BD20522056
:10009000C30B4728432818211F151F194D281E0878
:1000A000A1000800A22020080A3C0318080005153A
:1000B000A82020081E3C0318A2280511152185152B
:1000C000A8202008323C0318A22885111521061407
:1000D000A8202008463C0318A228061015218614E3
:1000E000A82020085A3C0318A228861015210615BE
:1000F000A82020086E3C0318A22806111521861599
:10010000A8202008823C0318A22886111521061673
:10011000A8202008963C0318A2280612152186164E
:10012000A8202008AA3C0318A2288612152105172A
:10013000A8202008BE3C0318A22805131521851706
:10014000A8200800860105118511051385130800F4
:100150001E211E21080022210800A220AB2002300F
:10016000A400CC308500FF3086002221A22022216D
:10017000A40BB128AB20A22008000A30C30008005D
:100180003230C30008002830C40008009F154B20FF
:100190009F112108A2004B20A22022212221C02051
:1001A000D620C30BD0282221222108000515A82023
:1001B0000511A50122088F3C031811292208973C3C
:1001C0000318092925142208993C03180D29251024
:1001D000A5142208A03C03180D29A51025152208F6
:1001E000A63C03180D292511A5152208AD3C0318BE
:1001F0000D29A51125162208B93C03180D29251231
:10020000A5162208C23C03180D290517A8200513BE
:1002100011298515A8208511112925088600A820F7
:1002200086018517A820851308000130C1001A290E
:100230003230C1000000C10B1A2908000230242905
:1002400014302429C8302429C000F930C10000002E
:0A025000C10B2729C00B2529080067
:02400E00383F39
:02401000FC3F73
:00000001FF
